:100000000C94280018950000189500001895000021
:10001000189500001895000018950000189500002C
:10002000189500000C94AB09189500001895000075
:10003000189500001895000018950000189500000C
:1000400018950000189500001895000018950000FC
:100050008FE181BD87E181BD8FE58DBFC4E0E8E719
:100060004E2E88E08EBFD8E0F7E05F2EEEEFF7E08F
:10007000A0E6B0E088278D933197E9F783E389B94B
:1000800088E18AB9662481E48ABB81E38BBB8FEB6C
:1000900087BB8FEB88BB88E084BB83E085BB80E0B7
:1000A00081BB8BE382BB80E08FBD81E08EBD8FE1A1
:1000B00081BD87E181BD86E086B980E487B9C398B8
:1000C000C29AD89ADE9AC498C798C598F894A89509
:1000D0007091CE007F7E7093CE007091CE00777FBE
:1000E0007093CE000E94CC127091CE007064709319
:1000F000CE00EFEFF1E0A0ECB0E091E00E94CB2960
:100100000091C000003081E009F080E08F93009101
:10011000C0000E3F80E010F009F081E09F91892B34
:10012000882311F40C9497008EEB8093C00000910B
:10013000C0004AE0040F01BF89E190E00E94452819
:10014000ECEEF3E50E948C270027AEECB0E08C913A
:1001500084FB0EF401E041E0041711F00C94B800A8
:10016000E6E0F4E50E948C270E9498270C94CB00CF
:10017000E8E0F4E50E948C27AEECB0E08C9183FBC4
:10018000A8E6B7E00E94A6288D9388278C930E944A
:1001900084270E949827EAE0F0E0BB27A0E10E94B4
:1001A000C8290F3211F40C940B01EBE0F0E0A0E150
:1001B000BB278FE08C937BE70E94B729ECE0F0E04F
:1001C00001E010E0A0E1BB277BE70E94B929EAE04B
:1001D000F0E0A0E1BB278FE28C937BE70E94B72978
:1001E000EEE0F0E0A0E1BB2780E18C937BE70E948A
:1001F000B729E0E1F0E000E010E0A0E1BB277BE7F9
:100200000E94B929EFE0F0E0A0E1BB2780E08C93E9
:100210007BE70E94B729EBE0F0E0ABEBB0E00E9497
:10022000C8290091BB00043618F011F00C941A0193
:100230000C941D0184E68093BB0080E797E9ACEB4A
:10024000B0E08D939C93ECE0F0E0A5EBB0E00E9471
:10025000CA2980E08093D00080E08093C10080E0D4
:100260008093C2000E942A0BE0E1F0E0A3E6B0E038
:100270000E94CA29A3E6B0E00E940727E0E1F0E06F
:10028000A3E6B0E07BE70E94B929A5EBB0E00D91B1
:100290001C91003050E0150711F00C94550181E0DD
:1002A00090E0A5EBB0E08D939C93EAE0F4E50E942A
:1002B0008C27A8E6B7E0EBEBF0E00E9414290E943F
:1002C0008427E2E1F4E50E948C27A8E6B7E0E1ECA0
:1002D000F0E00E9414290E948427E2E1F4E50E94E4
:1002E0008C27A8E6B7E0E2ECF0E00E9414290E9417
:1002F0008427E2E1F4E50E948C27A8E6B7E0E5EB6D
:10030000F0E00E9405290E948427E2E1F4E50E94C2
:100310008C27A8E6B7E0E3E6F0E00E9405290E94FA
:1003200084270E94982780E08093CD007091B700C9
:100330007F7E7093B70086E08093BE008DE080934F
:10034000BF0084E190E00E944528DE980E94312899
:10035000C49AE4E1F4E50E948C270E94982788EC77
:1003600090E00E944528A89581B5886181BD877F6E
:1003700081BDE0E6F0E0FA93EA930E94841C2296A5
:10038000A89500916000003011F40C94D3010E94F4
:10039000D012EEE1F4E50E948C270E9498270E947B
:1003A000EE0A0C94D8017091CE007F777093CE0046
:1003B000E8E2F4E50E948C270E942C1384E690E08A
:1003C0000E9445280027AEECB0E08C9187FB0EF42C
:1003D00001E040E0041711F00C94F0010E94981322
:1003E0000E94D60B8FEF0E949B2782E390E00E9431
:1003F00045287894A89581B5886081BDA1EBB0E0CF
:100400004D915C91A5EBB0E00D911C91041715077F
:1004100018F011F00C940E020C94140281E090E09C
:10042000A5EBB0E08D939C930027A7EBB0E08C91F7
:1004300085FB0EF401E041E0041781E009F080E063
:100440008F930027AEECB0E08C9187FB0EF401E0B7
:1004500040E0041781E009F080E09F9189238F93A9
:100460000027A7EBB0E08C9180FB0EF401E040E0A8
:10047000041781E009F080E09F918923882311F41B
:100480000C945502E5EBF0E0FA93EA935A924A9203
:1004900080E0A42DB52D8C9381E00E94F4260E946B
:1004A000580F249681E00E94F02680E08093B800E7
:1004B00080E08093690080E08093D20080E08093A8
:1004C000CF00A895AAE6B0E088278C930027AEEC71
:1004D000B0E08C9187FB0EF401E041E0041711F0CD
:1004E0000C9474020E94CC120091CD00003081E087
:1004F00009F080E08F930027A7EBB0E08C9182FB9E
:100500000EF401E041E0041781E009F080E09F91E2
:10051000892B882311F40C942803E0E6F0E0FA9389
:10052000EA930E94D41122964091D200009160007B
:10053000041711F40C942803809160008093D2007A
:1005400000916000003011F40C9428038091D000D9
:100550008093CF000091D100003011F00C94FE0286
:1005600000916000013011F00C94BE0281E090E037
:10057000A5EBB0E08D939C930C94E002023011F057
:100580000C94CA0282E090E0A5EBB0E08D939C93BE
:100590000C94E002043011F00C94D60283E090E059
:1005A000A5EBB0E08D939C930C94E002083011F021
:1005B0000C94E00284E090E0A5EBB0E08D939C9376
:1005C0000027A7EBB0E08C9185FB0EF401E041E041
:1005D000041781E009F080E08F93009160000830FB
:1005E00081E009F080E09F918923882311F40C9425
:1005F000FC0281E08093CF000C942203A0E6B0E0DF
:100600008C91A5EBB0E08D9388278C930027A7EB06
:10061000B0E08C9185FB0EF401E041E0041781E02D
:1006200009F080E08F93009160000F3081E009F0C5
:1006300080E09F918923882311F40C94220381E0A8
:100640008093CF00AAE6B0E0E2E3F4E50E946B27D6
:1006500080E0809369000027A7EBB0E08C9181FBDC
:100660000EF401E040E0041711F00C94CD03E9E62C
:10067000F0E0FA93EA930E947C11229600916900BF
:10068000043011F00C9446030E94BF0A00916900E7
:10069000013011F00C945203AAE6B0E0E4E3F4E573
:1006A0000E946B2780E08093600000916900023017
:1006B00081E009F080E08F930091BB00043681E077
:1006C00008F080E09F918923882311F40C94700333
:1006D000ABEBB0E08C918B5F8C9381E080936000FA
:1006E00000916900033081E009F080E08F93009170
:1006F000BB00053081E009F080E09F9189238823C9
:1007000011F40C94890381E08093BB0081E0809315
:10071000600000916900033081E009F080E08F9370
:100720000091BB00053080E010F009F081E09F915E
:100730008923882311F40C94A503ABEBB0E08C91D2
:1007400085508C9381E080936000009160000130BF
:1007500011F00C94CD038EB5887F8EBD5A924A92CB
:100760008091BB00A42DB52D8C9381E00E94F426CE
:100770000E947223229681E00E94F026EBE0F0E0D6
:10078000ABEBB0E07BE70E94B7290091CD000130D0
:1007900011F00C94CD0381E08EBDEAE6F0E0AAE60C
:1007A000B0E00E949A28AAE6B0E08C91803081E007
:1007B00009F480E08F9300916900003081E009F432
:1007C00080E09F91892B8F930091B800013081E0E8
:1007D00009F080E09F91892B882311F40C94610229
:1007E0000091B800013011F00C941F0480E0809358
:1007F000B800AAE6B0E0E4E3F4E50E946B27002726
:10080000A7EBB0E08C9180FB0EF401E041E004170F
:1008100011F00C941104AAE6B0E0E2E3F4E50E94C2
:100820006B270091CF00003018F011F00C941A04DF
:100830000C941F048091CF008A958093CF00AAE684
:10084000B0E0E2E3F4E50E94E22911F00C94910497
:100850000091CD00013011F00C9430040E94BF0AC9
:10086000A1EBB0E04D915C91A5EBB0E00D911C9136
:100870000417150718F011F00C948C040027AEEC47
:10088000B0E08C9187FB0EF401E040E0041711F01A
:100890000C945D04E5EBF0E0FA93EA935A924A92E5
:1008A00080E0A42DB52D8C9381E00E94F4260E9457
:1008B000580F249681E00E94F0260027AEECB0E0AD
:1008C0008C9187FB0EF401E041E0041711F00C94C9
:1008D0008A040E94EE0A0027AEECB0E08C9187FB00
:1008E0000EF401E040E0041711F00C948A04E5EBEB
:1008F000F0E0FA93EA935A924A9280E0A42DB52D43
:100900008C9381E00E94F4260E94580F249681E087
:100910000E94F0260C948F0480E08093D2000C9407
:100920006609E6E3F4E50E94E22911F00C949F04C5
:100930000E94BF0A80E08093D2000C946609E8E32D
:10094000F4E50E94E22911F00C94D9040091CD0045
:10095000013011F00C94D7040027A7EBB0E08C9184
:1009600084FB0EF401E040E0041711F00C94C9047C
:100970008EB5887F8EBD89B78B7F89BF7091B70098
:1009800070617093B70084E690E00E9445280C9453
:10099000D7047091B7007F7E7093B70080E29EE429
:1009A0009DBD8CBD81E08EBD89B7846089BF0C94EC
:1009B0006609E4E3F4E50E94E22911F00C94710564
:1009C0000091CD00013011F00C94E8040E94BF0AA0
:1009D000A5EBB0E00E9407270027AEECB0E08C91B9
:1009E00086FB0EF401E041E0041711F00C940D05B4
:1009F0000027A7EBB0E08C9185FB0EF401E040E00E
:100A0000041711F00C940805A5EBB0E00E940D2727
:100A10007091CE007F7B7093CE00A1EBB0E04D9142
:100A20005C91A5EBB0E00D911C910417150718F02F
:100A300011F00C941D050C94230581E090E0A5EBCA
:100A4000B0E08D939C930027AEECB0E08C9187FBD7
:100A50000EF401E040E0041711F00C944205E5EBC0
:100A6000F0E0FA93EA935A924A9280E0A42DB52DD1
:100A70008C9381E00E94F4260E94580F249681E016
:100A80000E94F0260027AEECB0E08C9187FB0EF4BC
:100A900001E041E0041711F00C946F050E94EE0A8A
:100AA0000027AEECB0E08C9187FB0EF401E040E053
:100AB000041711F00C946F05E5EBF0E0FA93EA935C
:100AC0005A924A9280E0A42DB52D8C9381E00E9429
:100AD000F4260E94580F249681E00E94F0260C9480
:100AE0006609EAE3F4E50E94E22911F00C94E905B5
:100AF0000091CD00013011F00C9480050E94BF0AD6
:100B0000A5EBB0E00D911C91013050E0150718F0F5
:100B100011F00C948D050C949305A5EBB0E00E94A8
:100B20000D270C949B05A1EBB0E08D919C91A5EB5A
:100B3000B0E08D939C930027AEECB0E08C9187FBE6
:100B40000EF401E040E0041711F00C94BA05E5EB57
:100B5000F0E0FA93EA935A924A9280E0A42DB52DE0
:100B60008C9381E00E94F4260E94580F249681E025
:100B70000E94F0260027AEECB0E08C9187FB0EF4CB
:100B800001E041E0041711F00C94E7050E94EE0A21
:100B90000027AEECB0E08C9187FB0EF401E040E062
:100BA000041711F00C94E705E5EBF0E0FA93EA93F3
:100BB0005A924A9280E0A42DB52D8C9381E00E9438
:100BC000F4260E94580F249681E00E94F0260C948F
:100BD0006609ECE3F4E50E94E22911F00C945C064E
:100BE000A5EBB0E00E940727A1EBB0E04D915C912E
:100BF000A5EBB0E00D911C910417150718F011F04A
:100C00000C9404060C940A0681E090E0A5EBB0E099
:100C10008D939C938EB5887F8EBDA1E7B0E00D913A
:100C20001D912D913C91A1E9B0E00D931D932D9361
:100C30003C930027AEECB0E08C9187FB0EF401E012
:100C400040E0041711F00C9452065A924A92A1E91E
:100C5000B0E00D911D912D913C91A42DB52D0D93DA
:100C60001D932D933C9384E00E94F4265A924A925D
:100C7000A5EBB0E08D919C91A42DB52D8D939C9307
:100C800082E00E94F4265A924A9280E0A42DB52D6B
:100C90008C9381E00E94F4260E94A714269687E098
:100CA0000E94F0260091CD00013011F00C945A06FC
:100CB00081E08EBD0C946609E8E0F4E50E94E2292B
:100CC00011F00C94D006A5EBB0E00D911C91013011
:100CD00050E0150718F011F00C9470060C9476068D
:100CE000A5EBB0E00E940D270C947E06A1EBB0E0CE
:100CF0008D919C91A5EBB0E08D939C938EB5887FF0
:100D00008EBDA1E7B0E00D911D912D913C91A1E91F
:100D1000B0E00D931D932D933C930027AEECB0E013
:100D20008C9187FB0EF401E040E0041711F00C9465
:100D3000C6065A924A92A1E9B0E00D911D912D91FB
:100D40003C91A42DB52D0D931D932D933C9384E0E0
:100D50000E94F4265A924A92A5EBB0E08D919C91A4
:100D6000A42DB52D8D939C9382E00E94F4265A9277
:100D70004A9280E0A42DB52D8C9381E00E94F42648
:100D80000E94A714269687E00E94F0260091CD00CD
:100D9000013011F00C94CE0681E08EBD0C946609F2
:100DA000EEE3F4E50E94E22911F00C94E006ECE099
:100DB000F0E0A5EBB0E07BE70E94B9290C9466094E
:100DC000E0E4F4E50E94E22911F00C94F4060E949C
:100DD000BF0A8DE181BD85E181BD81B5886081BD9E
:100DE0000C94F0060C946609AAE6B0E0E2E4F4E59F
:100DF0000E94E22981E008F480E08F93AAE6B0E047
:100E0000E4E4F4E50E94E22981E010F009F080E0DA
:100E10009F918923882311F40C94C80789B78B7F8D
:100E200089BF8EB5887F8EBD0E947827A0E6B0E08E
:100E30008C9300916000003011F40C9414070E9410
:100E40007C27A5EBB0E08D9388278C9380E080937E
:100E5000CD007091B7007F7E7093B700A1EBB0E03A
:100E60004D915C91A5EBB0E00D911C910417150715
:100E700080E010F009F081E08F93A5EBB0E00D91D8
:100E80001C91003050E0150781E009F080E09F914F
:100E9000892B882311F40C94680781E090E0A5EB7E
:100EA000B0E08D939C93E5EBF0E0FA93EA935A92CD
:100EB0004A9281E0A42DB52D8C9381E00E94F42606
:100EC0000E94580F249681E00E94F0260C94C607D9
:100ED0000027AEECB0E08C9187FB0EF401E040E01F
:100EE000041781E009F080E08F93AAE6B0E0E2E425
:100EF000F4E50E94E22981E009F080E09F918923D6
:100F0000882311F40C949707E5EBF0E0FA93EA9349
:100F10005A924A9281E0A42DB52D8C9381E00E94D3
:100F2000F4260E94580F249681E00E94F0260027A4
:100F3000AEECB0E08C9187FB0EF401E040E00417CA
:100F400081E009F080E08F93AAE6B0E0E4E4F4E504
:100F50000E94E22981E009F080E09F9189238823A3
:100F600011F40C94C607E5EBF0E0FA93EA935A9279
:100F70004A9280E0A42DB52D8C9381E00E94F42646
:100F80000E94580F249681E00E94F0260C94660976
:100F9000E6E4F4E50E94E22911F00C9403080E94B3
:100FA0007827A0E6B0E08C9300916000003011F447
:100FB0000C94CF070E947C27ABEBB0E08C938EB5EE
:100FC000887F8EBD5A924A928091BB00A42DB52D88
:100FD0008C9381E00E94F4260E947223229681E085
:100FE0000E94F026EBE0F0E0ABEBB0E07BE70E9484
:100FF000B7290091CD00013011F00C94010881E077
:101000008EBD0C946609E8E4F4E50E94E22911F033
:101010000C9451080E947827A0E6B0E08C930091D0
:101020006000003011F40C940A088091C100809394
:1010300060000E947C27A1ECB0E08C93A1ECB0E0B2
:101040008C918F738C930E942A0B0091C10040E118
:101050000423A0E6B0E00C9300916000003111F091
:101060000C9436080E94CC120C9438080E94CE12C0
:10107000A1ECB0E08C918F7E8C938EB5887F8EBD75
:10108000EEE0F0E0A1ECB0E07BE70E94B729009130
:10109000CD00013011F00C944F0881E08EBD0C940E
:1010A0006609E6E0F4E50E94E22911F00C94B50827
:1010B0000091C1004FE30423A0E6B0E00C9300913F
:1010C000CD00013011F00C946A08A0E6B0E08C91DC
:1010D00080588C930027AEECB0E08C9187FB0EF427
:1010E00001E041E0041711F00C947B08A0E6B0E0A9
:1010F0008C91805C8C930027A7EBB0E08C9184FBF3
:101100000EF401E041E0041711F00C948C08A0E605
:10111000B0E08C91805E8C938091B50080936200EA
:101120008EB5887F8EBD31E0A0E6B0E00E949327A7
:1011300031E0ABEBB0E00E94932731E0A2E6B0E0F3
:101140000E9493278091B1008093620031E0A2E673
:10115000B0E00E9493270091CD00013011F00C9473
:10116000B30881E08EBD0C946609EAE4F4E50E94C0
:10117000E22911F00C943809A7EDB0E00D911D9112
:101180002D913C91A3EDB0E04D915D916D917C91DD
:101190000E94ED28A5E6B0E00D931D932D933D939D
:1011A000A5E6B0E00E94F826A5E6B0E00D911D91FD
:1011B0002D913C9140E052E060E070E00E94A52754
:1011C000A5E6B0E00D931D932D933D93A5E6B0E009
:1011D0000D911D912D913C91A3ECB0E04C915527C0
:1011E000662777270E94AA27A5E6B0E04D935D9376
:1011F0006D937D93A5E6B0E00D911D912D913C91ED
:101200004AE050E060E070E00E94AA27A5E6B0E066
:101210004D935D936D937D9344E150E060E070E009
:10122000A5E6B0E00D911D912D913C910E94F22810
:101230000CF402C00C94260900E010E020E030E03D
:10124000A5E6B0E00D931D932D933C938EB5887F5A
:101250008EBD34E0A5E6B0E00E9493270091CD005A
:10126000013011F00C94360981E08EBD0C946609B2
:10127000ECE4F4E50E94E22911F00C9450098EB5DB
:10128000887F8EBDA3EAB0E00E9486270091CD0042
:10129000013011F00C944E0981E08EBD0C9466096A
:1012A000EEE4F4E50E94E22911F00C9466098EB593
:1012B000887F8EBD0E9443140091CD00013011F053
:1012C0000C94640981E08EBD0C94660981E090E085
:1012D0000E94452800916900003018F011F00C942C
:1012E00073090C94A909A895E0E6F0E0FA93EA9353
:1012F0000E947C11229600916000043011F00C9441
:101300008F090E94BF0A80E08093D2000E94CE1213
:1013100085E090E00E94452880E080936000009185
:10132000CD00003011F00C94990985E090E00E9406
:10133000452800916000003011F00C947309009171
:10134000CD00003011F00C94A90985E090E00E94D6
:1013500045280C9461020F921F922F923F924F9258
:101360005F927F928F929F92AF92BF920F931F9343
:101370002F933F934F935F936F937F938F939F939D
:10138000AF93BF93CF93DF93EF93FF938FB78F9379
:10139000F89489B78B7F89BF8EB5887F8EBD5A92AE
:1013A0004A9280E092E0A42DB52D8D939C9382E02B
:1013B0000E94F4260E946E26229682E00E94F02669
:1013C0000091DB000A3011F00C94E8090E94CC1265
:1013D0000E94B81F0091DB000A3011F00C94F5094F
:1013E0000E94CE1280E08093DB00ABEDB0E08C91E8
:1013F0008F5F8C93A8950027AEECB0E08C9187FBB3
:101400000EF401E040E0041711F00C941A0A5A920D
:101410004A9280E092E0A42DB52D8D939C9382E0BA
:101420000E94F4260E946E26229682E00E94F026F8
:101430000E94B81FA7EDB0E04D915D916D917C9138
:10144000A3EDB0E00D911D912D913C910E94F228E9
:1014500080E00CF481E08F930027AEECB0E08C913B
:1014600087FB0EF401E040E0041781E009F080E022
:101470009F918923882311F40C94490A80E49CE904
:101480009DBD8CBD81E08EBD89B7846089BF0C9401
:101490009F0A80E08093CD007091B7007F7E7093AB
:1014A000B7000027AEECB0E08C9187FB0EF401E0B2
:1014B00040E0041781E009F080E08F930091CF00B5
:1014C000013081E009F480E09F918923882311F4A1
:1014D0000C94730AA7EBB0E08C9185FBA8EBB0E00D
:1014E000882780F98C930091C1004FE70423A1E67F
:1014F000B0E00C930E94CE1280E08093D2000027CF
:10150000AEECB0E08C9184FB0EF401E041E00417F6
:1015100081E009F080E08F930027AEECB0E08C9181
:1015200083FB0EF401E041E0041781E009F080E064
:101530009F91892B882311F40C949F0ADC988F913A
:101540008FBFFF91EF91DF91CF91BF91AF919F91AD
:101550008F917F916F915F914F913F912F911F914B
:101560000F91BF90AF909F908F907F905F904F9022
:101570003F902F901F900F901895F894FFCF89B748
:101580008B7F89BF8EB5887F8EBD80E08093CD0034
:101590007091B7007F7E7093B7000027AEECB0E08B
:1015A0008C9184FB0EF401E041E0041781E009F026
:1015B00080E08F930027AEECB0E08C9183FB0EF4BB
:1015C00001E041E0041781E009F080E09F91892B60
:1015D000882311F40C94ED0ADC980895DE9A6E9835
:1015E000C498C598C7980E94CE12E2E0F0E00E942D
:1015F0009F27DE98C49A0E94312884E690E00E94DA
:101600004528A8957091CE007F777093CE00E0E6D4
:10161000F0E0FA93EA930E94841C22960091600005
:10162000003011F40C94240B7091CE00706870930C
:10163000CE0084E690E00E944528DE9A6E98C49819
:10164000C598C7980C94260B0E94981380E080934D
:10165000D200089581E00E9454287091B7007F7DE8
:101660007093B7000091C10041E00423A881B981C3
:101670000C93A881B9810C91003011F40C94450BA6
:101680007091B70070627093B7007091B7007E7F61
:101690007093B7000091C10042E00423A881B98192
:1016A0000C93A881B9810C91003011F40C945D0B5E
:1016B0007091B70071607093B7007091B7007D7F33
:1016C0007093B7000091C10044E00423A881B98160
:1016D0000C93A881B9810C91003011F40C94750B16
:1016E0007091B70072607093B7007091B7007B7F04
:1016F0007093B7000091C10048E00423A881B9812C
:101700000C93A881B9810C91003011F40C948D0BCD
:101710007091B70074607093B7007091B7007F7BD1
:101720007093B7000091C10040E20423A881B98101
:101730000C93A881B9810C91003011F40C94A50B85
:101740007091B70070647093B7007091CE007F7D88
:101750007093CE000091C20041E00423A881B981BA
:101760000C93A881B9810C91003011F40C94BD0B3D
:101770007091CE0070627093CE000091C20042E082
:101780000423A881B9810C93A881B9810C9142E00E
:101790000E94D2290C93A881B9818C918093D100A9
:1017A00081E0481A8827580A2296089582E00E940C
:1017B000542881E00E94542882E00E945428E0E5E9
:1017C000F4E50E948C270E94982780E0AA81BB81C3
:1017D0008C9383E4ABE9B0E08C938FE4ACE9B0E0A8
:1017E0008C938EE4ADE9B0E08C9386E4AEE9B0E092
:1017F0008C9389E4AFE9B0E08C93A7EBB0E08C91D7
:1018000086FBACEDB0E0882780F98C93A1EBB0E0CB
:101810008D919C91A881B9818D939C937091B70013
:1018200070647093B700A1E7B0E00D911D912D9108
:101830003C91A1E9B0E00D931D932D933C935A92F6
:101840004A92A1E9B0E00D911D912D913C91A42DFA
:10185000B52D0D931D932D933C9384E00E94F426A7
:101860005A924A9280E090E0A42DB52D8D939C93DE
:1018700082E00E94F4265A924A9281E0A42DB52D6E
:101880008C9381E00E94F4260E94A714269687E09C
:101890000E94F0268FE00E945428E3EAF0E006E080
:1018A000A881B9810E94A929A881B981EEE5F4E552
:1018B0000E94E2290FB68FE0481A8827580A22961C
:1018C0000FBE11F00C94800C81E0AA81BB818C9337
:1018D000E6E6F4E50E948C270E949827A1E9B0E093
:1018E0000D911D912D913C91A3EDB0E00D931D93B1
:1018F0002D933C930E94B81F0E94E00C0C94860C20
:10190000E4E7F4E50E948C270E949827ACEDB0E054
:101910008C9180FBA7EBB0E08C9186F98C93A5E7C6
:10192000B0E00D911D912D913C91A1E7B0E00D9398
:101930001D932D933C93A1E7B0E00D911D912D9146
:101940003C91A1E9B0E00D931D932D933C935A92E5
:101950004A92A1E9B0E00D911D912D913C91A42DE9
:10196000B52D0D931D932D933C9384E00E94F42696
:101970005A924A9280E090E0A42DB52D8D939C93CD
:1019800082E00E94F4265A924A9280E0A42DB52D5E
:101990008C9381E00E94F4260E94A714269687E08B
:1019A0000E94F026A881B9818D919C91A1EBB0E0B5
:1019B0008D939C9385E0481A8827580A26960895A7
:1019C00081E00E94542881E00E94542881E00E9416
:1019D000542882E00E94542882E00E94542882E029
:1019E0000E94542882E00E94542882E00E945428D9
:1019F00080E092E0AA81BB818D939C9380E0AA85D0
:101A0000BB858C9381E090E0AC81BD818D939C93EC
:101A1000AC81BD818D919C91A885B9858D939C9356
:101A2000AA81BB814D915C91A885B9850D911C91CE
:101A30000417150718F011F00C94340DA885B9851A
:101A4000AD90BC90A7EFB0E0AA0DBB1D0C910D307E
:101A500011F00C942D0D0C94340DA885B9850E94BD
:101A6000072711F00C94100DA885B985AD90BC9096
:101A7000A8EFB0E0AA0DBB1D0C910A3011F00C9438
:101A80004D0DA885B9850D911C9141E050E0040FE2
:101A9000151FA885B9850D931C93A7EEB0E0882784
:101AA0008C93AC81BD810D911C91A885B9854D9118
:101AB0005C91040F151FAE81BF810D931C93AC8107
:101AC000BD818D919C91A881B9818D939C93AE81AC
:101AD000BF814D915C91A881B9810D911C91041732
:101AE000150718F011F00C94CD0D81E00E945428D8
:101AF000AA81BB81AD90BC90A7EFB0E0AA0DBB1D41
:101B00008C91A881B9818D9388278C93A881B98104
:101B1000EEE7F4E50E94E2290FB681E0481A882733
:101B2000580A22960FBE11F00C94980D0C94CD0D0E
:101B3000A881B981AD90BC90A7EFB0E0AA0DBB1D04
:101B40000C910D3011F00C94A70D0C94CD0DA881C3
:101B5000B981AD90BC90A7EFB0E0AA0DBB1D0C9170
:101B6000003211F40C94C60DA881B981AD90BC90DF
:101B7000A7EFB0E0AA0DBB1D8C91A7EEB0E08F934C
:101B80000E9471278F918D9388278C93A881B981AA
:101B90000E94072711F00C94670DA7EEB0E08C911E
:101BA000803011F40C942E0FE7EEF0E0A7EEB0E0D9
:101BB0000E94A02982E10E945428E7EEF0E001E0B3
:101BC000A881B9810E94A929A881B981E0E8F4E53A
:101BD0000E94E2290FB682E1481A8827580A229605
:101BE0000FBE11F00C942E0FA7EEB0E0E2E8F4E582
:101BF0002FEF91E00E945F28AE85BF850C93AE85E4
:101C0000BF850C91003018F011F00C94090E0C9463
:101C10002E0FAE85BF858C9182508C9382E0E7EECB
:101C2000F0E0AE85BF850C910A93ADEDB0E00E9467
:101C3000A229EDEDF0E0ADEDB0E00E948E28AE857A
:101C4000BF858C918C5F8C93AE85BF858C91E7EEC0
:101C5000F0E00FEF0A93A2EEB0E00E94A229A2EEFC
:101C6000B0E00E945E29AC85BD850C93ADEDB0E07F
:101C7000E6E8F4E50E94E22911F00C94540EAC85DC
:101C8000BD858C918093BB00EAE8F4E50E948C2727
:101C9000A8E6B7E0EC85FD850E9414290E94842700
:101CA0000E9498270C942E0FE2E9F4E50E94E229A5
:101CB00011F00C94700EAC85BD858C918093D10091
:101CC000E6E9F4E50E948C27A8E6B7E0EC85FD85FF
:101CD0000E9414290E9484270E9498270C942E0F9A
:101CE000EEE9F4E50E94E22911F00C94900EAC8527
:101CF000BD858C9180FBA7EBB0E08C9181F98C9332
:101D0000E2EAF4E50E948C27A8E6B7E0EC85FD85C1
:101D10000E9414290E9484270E9498270C942E0F59
:101D2000EAEAF4E50E94E22911F00C94AC0EAC85CD
:101D3000BD858C918093DC00EEEAF4E50E948C274F
:101D4000A8E6B7E0EC85FD850E9414290E9484274F
:101D50000E9498270C942E0FE8EBF4E50E94E229EC
:101D600011F00C94CC0EAC85BD858C9180FBA7EB5B
:101D7000B0E08C9182F98C93ECEBF4E50E948C2717
:101D8000A8E6B7E0EC85FD850E9414290E9484270F
:101D90000E9498270C942E0FE8ECF4E50E94E229AB
:101DA00011F00C94EC0EAC85BD858C9180FBA7EBFB
:101DB000B0E08C9185F98C93ECECF4E50E948C27D3
:101DC000A8E6B7E0EC85FD850E9414290E948427CF
:101DD0000E9498270C942E0FE2EDF4E50E94E22970
:101DE00011F00C94140FE6EDF4E50E948C27A8E6A0
:101DF000B7E0EC85FD850E9414290E9484270E948B
:101E000098277091B70071607093B700AC85BD855D
:101E10000C91013011F00C94120F7091B7007E7F7D
:101E20007093B7000C942E0FECEDF4E50E94E229BC
:101E300011F00C942E0FE0EEF4E50E948C27A8E63A
:101E4000B7E0EC85FD850E9414290E9484270E943A
:101E50009827AC85BD858C918093D000A885B985E5
:101E60000D911C9141E050E0040F151FAC81BD8124
:101E70000D931C93AA81BB814D915C91AC81BD8176
:101E80000D911C910417150710F40C944B0F81E071
:101E9000AA85BB858C93AA85BB850C91013011F076
:101EA0000C94080D8DE0481A8827580A609608950A
:101EB00082E00E94542881E00E94542881E00E9420
:101EC00054288EB5887F8EBD7091B7007F7E709349
:101ED000B700A1E7B0E00D911D912D913C91A1E9D2
:101EE000B0E00D931D932D933C935A924A92A1E931
:101EF000B0E00D911D912D913C91A42DB52D0D9328
:101F00001D932D933C9384E00E94F4265A924A92AA
:101F1000AC85BD858D919C91A42DB52D8D939C9301
:101F200082E00E94F4265A924A9280E0A42DB52DB8
:101F30008C9381E00E94F4260E94A714269687E0E5
:101F40000E94F026A3EAB0E0E6EEF4E52FEF91E080
:101F50000E945F28002F003011F00C94B90F00E0B0
:101F600010E020E030E0ADE8B0E00D931D932D933C
:101F70003C9340E050E060E070E0ADE8B0E00D91EF
:101F80001D912D913C910E94F22811F00C94D30FD9
:101F9000A7EBB0E08C9185FBA8EBB0E0882780F937
:101FA0008C930C9476110E9426235A924A92809127
:101FB000BB00A42DB52D8C9381E00E94F4260E94D5
:101FC0007223229681E00E94F0265A924A92ACEB4C
:101FD000B0E08D919C91A42DB52D8D939C9382E0C2
:101FE0000E94F4260E940A24229682E00E94F02693
:101FF000A1E9B0E00D911D912D913C91A3EDB0E0D0
:102000000D931D932D933C93A1E9B0E00D911D918B
:102010002D913C91ADE8B0E04D915D916D917C9139
:102020000E94E828A7EDB0E00D931D932D933D93FA
:1020300080E0AA81BB818C9380E0A881B9818C93D8
:102040000E94B81FA881B9818C918F5F8C9381E029
:1020500090E0AC81BD818D939C93AC81BD810D914D
:102060001C910F3F51E0150718F011F00C94671008
:10207000AC81BD81AD90BC90A7EFB0E0AA0DBB1DB7
:102080000C910F3F81E009F080E08F93AC81BD811E
:10209000AD90BC90A8EFB0E0AA0DBB1D0C910F3E17
:1020A00080E010F009F081E09F918923882311F4EA
:1020B0000C94601081E0AA81BB818C930C94671012
:1020C000AC81BD810E94072711F00C942D10AA81CC
:1020D000BB810C91013081E009F080E08F93A881F1
:1020E000B9810C91003081E009F080E09F91892B4B
:1020F000882311F40C94201080E18093C300A88100
:10210000B9810C91003018F011F00C9489100C94E6
:102110003F11AC81BD81AD90BC90A9EFB0E0AA0D9C
:10212000BB1D8C91AC81BD818D9388278C93AC8134
:10213000BD810D911C9140E150E00E942527AC81AA
:10214000BD814D935C93AC81BD810D911C9101309B
:1021500050E0150711F00C94B21084E08093C30096
:102160000C943F11023050E0150711F00C94BD1093
:1021700085E08093C3000C943F11033050E01507B5
:1021800011F00C94C81086E08093C3000C943F11AA
:10219000043050E0150711F00C94D31087E08093C1
:1021A000C3000C943F11053050E0150711F00C945A
:1021B000DE1088E08093C3000C943F11063050E09D
:1021C000150711F00C94E9108AE08093C3000C9479
:1021D0003F11073050E0150711F00C94F4108CE01B
:1021E0008093C3000C943F11083050E0150711F0A4
:1021F0000C94FF108EE08093C3000C943F110930C3
:1022000050E0150711F00C940A1180E18093C3008F
:102210000C943F110A3050E0150711F00C94151181
:1022200084E18093C3000C943F110B3050E01507FC
:1022300011F00C94201188E18093C3000C943F119D
:102240000C3050E0150711F00C942B118CE18093A9
:10225000C3000C943F110D3050E0150711F00C94A1
:10226000361180E28093C3000C943F110E3050E091
:10227000150711F00C943F1188E28093C300AE81E2
:10228000BF810C91003011F00C94761181E08093A5
:10229000CD0088EC9FEA9DBD8CBD89B7846089BF65
:1022A00081E08EBD0027AEECB0E08C9184FB0EF493
:1022B00001E041E0041781E009F080E08F930027FE
:1022C000AEECB0E08C9183FB0EF401E041E004172A
:1022D00081E009F080E09F91892B882311F40C9410
:1022E0007211DC9A85E090E00E94452884E0481A4B
:1022F0008827580A2696089580E0A881B9818C9392
:102300000027BB27A0E38C9183FB0EF401E040E0A3
:10231000041711F00C94901182E0A881B9818C937C
:102320000027BB27A0E38C9184FB0EF401E040E082
:10233000041711F00C94A01181E0A881B9818C934D
:102340000027BB27A3E38C9181FB0EF401E040E062
:10235000041711F00C94B01183E0A881B9818C931B
:102360000027BB27A3E38C9181FB0EF401E040E042
:10237000041781E009F080E08F930027BB27A0E3DA
:102380008C9183FB0EF401E040E0041781E009F03A
:1023900080E09F918923882311F40C94D31184E069
:1023A000A881B9818C93089581E00E94542881E02E
:1023B0000E94542881E00E9454285398549880E049
:1023C00081BB909A919AEF93FF93E0EFF1E00E9426
:1023D0001928FF91EF9180E0AC81BD818C9300279B
:1023E000BB27A0E38C9180FB0EF401E040E00417D2
:1023F00011F00C94FF1181E0AC81BD818C9300271A
:10240000BB27A0E38C9181FB0EF401E040E00417B0
:1024100011F00C941012AC81BD818C918E5F8C9365
:102420000027BB27A9E38C9185FB0EF401E040E077
:10243000041711F00C942112AC81BD818C918C5F3A
:102440008C930027BB27A9E38C9184FB0EF401E059
:1024500040E0041711F00C943212AC81BD818C91D4
:10246000885F8C934091D200AC81BD810C910417A0
:1024700011F40C94BB1281E0A881B9818C93A881DE
:10248000B9810C91043018F011F00C94AC12009149
:10249000CD00003011F00C9451128AE090E00E94BF
:1024A000452880E0AA81BB818C930027BB27A0E34D
:1024B0008C9180FB0EF401E040E0041711F00C94C5
:1024C000651281E0AA81BB818C930027BB27A0E322
:1024D0008C9181FB0EF401E040E0041711F00C94A4
:1024E0007612AA81BB818C918E5F8C930027BB27CB
:1024F000A9E38C9185FB0EF401E040E0041711F094
:102500000C948712AA81BB818C918C5F8C930027DD
:10251000BB27A9E38C9184FB0EF401E040E0041793
:1025200011F00C949812AA81BB818C91885F8C93D6
:10253000AC81BD814C91AA81BB810C91041711F42F
:102540000C94A4120C94AC12A881B9818C918F5F69
:102550008C9311F00C943F12AC81BD814C91AA81F7
:10256000BB810C91041711F40C94BB128091D20022
:10257000AC81BD818C9381E081BB9198539A549A30
:10258000AC81BD818C91AE81BF818C9383E0481A70
:102590008827580A26960895AB980895AB9A08950F
:1025A00081E00E94542881E0A881B9818C93A881A0
:1025B000B9810C91063018F011F00C94F3120E94BE
:1025C000CC128FE090E00E9445280E94CE1284E653
:1025D00090E00E944528A881B9818C918F5F8C93EF
:1025E00011F00C94D71281E0481A8827580A2296D5
:1025F000089581E00E94542881E0A881B9818C93DC
:10260000AA81BB814C91A881B9810C91041718F063
:1026100011F00C9426135A924A9282E0A42DB52D03
:102620008C9381E00E94F4260E946424229681E02B
:102630000E94F0268DE790E00E944528A881B9818C
:102640008C918F5F8C9311F00C94001381E0481AE9
:102650008827580A229608950E943128C39A88EC48
:1026600090E00E94452881B5886081BD0E942623A4
:102670005A924A9281E0A42DB52D8C9381E00E945C
:10268000F4260E947223229681E00E94F02681B5F2
:10269000886181BD877F81BD84E690E00E944528E6
:1026A000FF27E0E1FA93EA935A924A928BE0A42D35
:1026B000B52D8C9381E00E94F4260E94FA25249681
:1026C00081E00E94F026013051E0150711F00C94D2
:1026D00082135A924A92ACEBB0E08D919C91A42D5A
:1026E000B52D8D939C9382E00E94F4260E940A24CB
:1026F000229682E00E94F026EAEEF4E50E948C2702
:102700000E9498275A924A9282E3A42DB52D8C9369
:1027100081E00E94F4260E947223229681E00E94AA
:10272000F026C29AD89A82E390E00E944528089544
:10273000A895A1E7B0E00D911D912D913C91A5E7E1
:10274000B0E00D931D932D933C93A1E7B0E00D9164
:102750001D912D913C91A1E9B0E00D931D932D9316
:102760003C935A924A92A1E9B0E00D911D912D91AE
:102770003C91A42DB52D0D931D932D933C9384E096
:102780000E94F4265A924A9280E090E0A42DB52D42
:102790008D939C9382E00E94F4265A924A9280E0A4
:1027A000A42DB52D8C9381E00E94F4260E94A714DD
:1027B000269687E00E94F026A895A1EBB0E00D9147
:1027C0001C91013050E0150710F00C940E145A9231
:1027D0004A9281E0A42DB52D8C9381E00E94F426CD
:1027E0000E946424229681E00E94F0268CE291E00F
:1027F0000E9445285A924A9280E0A42DB52D8C93D0
:1028000081E00E94F4260E946424229681E00E94C6
:10281000F0267091CE0070687093CE00A895A1E765
:10282000B0E00D911D912D913C91A1E9B0E00D9387
:102830001D932D933C93A5EBB0E00D911C910030BE
:1028400050E0150781E009F080E08F93A1EBB0E044
:102850004D915C91A5EBB0E00D911C91041715070B
:1028600080E010F009F081E09F91892B882311F41A
:102870000C94401481E090E0A5EBB0E08D939C9324
:102880000E94CE12089584E00E945428A3EDB0E087
:102890000D911D912D913C91A881B9810D931D93AE
:1028A0002D933C93A1E7B0E00D911D912D913C91AA
:1028B000A1E9B0E00D931D932D933C935A924A9257
:1028C000A1E9B0E00D911D912D913C91A42DB52D64
:1028D0000D931D932D933C9384E00E94F4265A920D
:1028E0004A928FE19EE4A42DB52D8D939C9382E0B6
:1028F0000E94F4265A924A9280E0A42DB52D8C9322
:1029000081E00E94F4260E94A714269687E00E9488
:10291000F026A1E7B0E00D911D912D913C91A1E928
:10292000B0E00D931D932D933C93A881B9810D9137
:102930001D912D913C91A3EDB0E00D931D932D932E
:102940003C9384E0481A8827580A2296089581E02B
:102950000E94542881E00E94542881E00E9454285B
:1029600080E090E0A3EBB0E08D939C937091B70072
:102970007F777093B70000E010E020E030E0ADE832
:10298000B0E00D931D932D933C930027A7EBB0E08F
:102990008C9186FB0EF401E041E0041781E009F020
:1029A00080E08F93A885B9850D911C91003050E08F
:1029B000150781E009F480E09F9189238F93AE8110
:1029C000BF810C91003081E009F080E09F91892364
:1029D000882311F40C944715A5E9B0E0E885F98542
:1029E0000E940529E5E9F0E0A8E6B7E00E949029F9
:1029F000E8E6F7E0A5E9B0E01127222704E0332755
:102A00000E94AA2881E4AC81BD818C93AC81BD81F8
:102A10008C9180939B0081E0E5E9F0E001E00A936E
:102A2000AAE6B0E00E94A229AAE6B0E08C91ACE947
:102A3000B0E08C9382E0E5E9F0E001E00A93AAE6D9
:102A4000B0E00E94A229AAE6B0E08C91ADE9B0E026
:102A50008C9383E0E5E9F0E001E00A93AAE6B0E0B8
:102A60000E94A229AAE6B0E08C91AEE9B0E08C9376
:102A700084E0E5E9F0E001E00A93AAE6B0E00E9414
:102A8000A229AAE6B0E08C91AFE9B0E08C9389B7B7
:102A90008B7F89BF8EB5887F8EBD81B5886181BDF2
:102AA000877F81BDA9ECB0E00D911D912D913C91E6
:102AB000A5ECB0E00D931D932D933C93A5E7B0E0FA
:102AC0004D915D916D917C91A1E7B0E00D911D91CB
:102AD0002D913C910E94F22811F00C94791502E09E
:102AE00010E020E030E0A5ECB0E00D931D932D93B5
:102AF0003C9380E0A881B9818C93EA81FB81FA93B1
:102B0000EA935A924A92AE85BF850D911D912D91FF
:102B10003C91A42DB52D0D931D932D933C9384E0F2
:102B20000E94F4260E94AF21249684E00E94F026A1
:102B3000AA81BB810C910E3F11F40C94AB157091DE
:102B4000CE0070687093CE007091B700706870937B
:102B5000B7000C94BE155A924A92AA85BB858D91F6
:102B60009C91A42DB52D8D939C9382E00E94F42618
:102B70000E94BF16229682E00E94F026A881B981A9
:102B80008C918F5F8C9340916E00A881B9810C91DC
:102B9000041781E009F080E08F930027A7EBB0E0F5
:102BA0008C9187FB0EF401E041E0041781E009F409
:102BB00080E09F918923882311F40C94741600916E
:102BC0007D000B3011F00C942116E5ECF0E0FA9347
:102BD000EA935A924A92A5ECB0E00D911D912D9185
:102BE0003C91A42DB52D0D931D932D933C9384E022
:102BF0000E94F4260E94FF1A249684E00E94F02688
:102C0000EA85FB85FA93EA935A924A92A5ECB0E0E2
:102C10000D911D912D913C91A42DB52D0D931D93DA
:102C20002D933C9384E00E94F4260E94951A2496EA
:102C300084E00E94F02680E0A881B9818C930C94F6
:102C40007216A5E7B0E04D915D916D917C91A1E781
:102C5000B0E00D911D912D913C910E94F22811F050
:102C60000C943816AA85BB850E94F8260C9472161F
:102C7000E5ECF0E0FA93EA935A924A92A5ECB0E0C0
:102C80000D911D912D913C91A42DB52D0D931D936A
:102C90002D933C9384E00E94F4260E94FF1A249610
:102CA00084E00E94F026EA85FB85FA93EA935A9223
:102CB0004A92A5ECB0E00D911D912D913C91A42D6F
:102CC000B52D0D931D932D933C9384E00E94F42623
:102CD0000E94951A249684E00E94F02680E0A88144
:102CE000B9818C930C947816AA85BB850E94F8262E
:102CF0000027A7EBB0E08C9187FB0EF401E041E0E8
:102D0000041711F00C947D15C49AA885B9850D910E
:102D10001C91003050E0150711F00C949716A3EBAE
:102D2000B0E08D919C91A1EBB0E08D939C930091CC
:102D3000CD00013081E009F080E08F930027AEECF8
:102D4000B0E08C9187FB0EF401E040E0041781E0D5
:102D500009F080E09F918923882311F40C94B9161F
:102D600080E593EC9DBD8CBD81E08EBD89B784600C
:102D700089BF83E0481A8827580A2696089584E078
:102D80000E94542884E00E94542881E00E94542824
:102D900081E00E94542881E00E94542881E00E9432
:102DA000542880E0AE81BF818C93AE81BF810C91AD
:102DB0000F3018F011F00C94A21881E0AC81BD81A5
:102DC0008C93AC81BD810C910C3018F011F00C94F7
:102DD00001178FEF0E9438280E943A280E94392854
:102DE000AC81BD81AD90BB24AFE7B0E0AA0DBB1DA7
:102DF0008C93AC81BD818C918F5F8C9311F00C947E
:102E0000E1168DE0AC81BD818C93AC81BD810C91CC
:102E1000043118F011F00C941F178FEF0E9438281E
:102E20000E943A280E943928A881B9818C93AC81EC
:102E3000BD818C918F5F8C9311F00C940517EA85FE
:102E4000FB85FA93EA93EA85FB85FA93EA930E945D
:102E50002A1924960027A7EBB0E08C9187FB0EF48B
:102E600001E041E0041711F00C9438170C949A1803
:102E700080E0AA81BB818C9300918B00003281E0BD
:102E800009F080E08F9300918B00003181E009F020
:102E900080E09F91892B882311F40C94531781E0D3
:102EA000AA81BB818C9300918000003081E009F4FD
:102EB00080E08F9300918000053E81E009F480E07E
:102EC0009F9189238F93AA81BB810C91013081E06E
:102ED00009F080E09F918923882311F40C948F18C6
:102EE00000918B00003211F00C947A17A3EBB0E044
:102EF0000E9407270027A7EBB0E08C9186FB0EF419
:102F000001E040E0041711F00C94AF1781E0AC81B0
:102F1000BD818C93AC85BD854D915C91A3EBB0E0F8
:102F20000D911C910417150781E009F080E08F9343
:102F3000A3EBB0E00D911C91003050E0150780E04C
:102F400010F009F081E09F918923882311F40C94FB
:102F5000AD1780E0AC81BD818C930C94E31780E0C9
:102F6000AC81BD818C9381E0A881B9818C93A881CB
:102F7000B9810C91053018F011F00C94E317A88179
:102F8000B981AD90BB24AAE9B0E0AA0DBB1D4C915C
:102F9000A881B981AD90BB24AFE7B0E0AA0DBB1DFD
:102FA0000C91041711F40C94DB1781E0AC81BD8106
:102FB0008C930C94E317A881B9818C918F5F8C93CB
:102FC00011F00C94B717AC81BD810C91003081E0F9
:102FD00009F080E08F93AC85BD850D911C910F3178
:102FE0005EE4150781E009F080E09F91892B88233A
:102FF00011F40C948F180E94BC18A885B9850D9106
:103000001D912D913C9140E052E060E070E00E9403
:10301000AA27ADE8B0E04D935D936D937D93E1E910
:10302000F0E0FA93EA935A924A92AE85BF850D91E9
:103030001D912D913C91A42DB52D0D931D932D9394
:103040003C9384E00E94F4260E94951A249684E022
:103050000E94F02680918B0080938C00AC85BD850A
:103060000D911C910F315EE4150711F00C9460185E
:10307000A8E6B7E0E3EBF0E00E9405290E94842770
:10308000EEEEF4E50E948C27A3EAB0E00E948627CA
:10309000EEEEF4E50E948C2700918B00003111F0D8
:1030A0000C945618E0EFF4E50E948C27A8E6B7E0F0
:1030B000E885F9850E9408290E9484270E949827A4
:1030C000AC81BD810C91003011F00C948F1870917F
:1030D000B70070687093B70000918C00003181E0F8
:1030E00009F080E08F93AC85BD850D911C910F3167
:1030F0005EE4150781E009F480E09F91892388232D
:1031000011F40C948F18AA85BB850D911D912D91FA
:103110003C91A9ECB0E00D931D932D933C9300914D
:103120008000003011F00C949A187091B70070680C
:103130007093B700AE81BF818C918F5F8C9311F03B
:103140000C94D5168FEF0E9438280E943A280E94CE
:103150003928A0E6B0E08C938FEF0E9438280E94B7
:103160003A280E943928A0E6B0E08C938CE0481AF7
:103170008827580A2C96089581E00E945428A3EAD3
:10318000B0E088278C9381E0A881B9818C93A881D5
:10319000B9810C91083018F011F00C94F618A88140
:1031A000B981AD90BB24AFE7B0E0AA0DBB1D0C9177
:1031B000003211F40C94EE18A881B981AD90BB24B3
:1031C000AFE7B0E0AA0DBB1D8C91A3EAB0E08F93EE
:1031D0000E9471278F918D9388278C93A881B98144
:1031E0008C918F5F8C9311F00C94C718A3EAB0E018
:1031F0000E947127E4EFF4E50E946B2789E0A88123
:10320000B9818C93A881B9810C910B3018F011F021
:103210000C942419A881B981AD90BB24AFE7B0E02C
:10322000AA0DBB1D8C91A3EAB0E08F930E94712779
:103230008F918D9388278C93A881B9818C918F5F12
:103240008C9311F00C94021981E0481A8827580ACF
:103250002296089581E00E94542881E00E9454281B
:1032600084E00E9454288FEF0E9438280E943A2858
:103270000E943928AC81BD818C938FEF0E94382841
:103280000E943A280E943928AA81BB818C93AA8186
:10329000BB810C9111272227332740E051E060E0E9
:1032A00070E00E94A527A885B9850D931D932D93E5
:1032B0003D93A885B9850D911D912D913C91AC81CF
:1032C000BD814C915527662777270E94E828A8855D
:1032D000B9850D931D932D933D93A885B9850D91C7
:1032E0001D912D913C9140E050E061E070E00E9422
:1032F000A527A881B9810D931D932D933D938FEF41
:103300000E9438280E943A280E943928AC81BD8149
:103310008C938FEF0E9438280E943A280E94392807
:10332000AC81BD818C938FEF0E9438280E943A288F
:103330000E943928AC81BD818C938FEF0E94382880
:103340000E943A280E943928AC81BD818C938FEF6E
:103350000E9438280E943A280E943928AC81BD81F9
:103360008C938FEF0E9438280E943A280E943928B7
:10337000AA81BB818C93AA81BB810C911127222742
:10338000332740E051E060E070E00E94A527A88567
:10339000B9850D931D932D933D93A885B9850D9106
:1033A0001D912D913C91AC81BD814C915527662793
:1033B00077270E94E828A885B9850D931D932D9342
:1033C0003D93A885B9850D911D912D913C91A881C2
:1033D000B9814D915D916D917C910E94E828A885FD
:1033E000B9850D931D932D933D938FEF0E9438283F
:1033F0000E943A280E943928AC81BD818C938FEFBE
:103400000E9438280E943A280E943928AA81BB814C
:103410008C93AA81BB810C9111272227332740E08E
:1034200051E060E070E00E94A527A881B9810D936A
:103430001D932D933D93A881B9810D911D912D91DF
:103440003C91AC81BD814C915527662777270E941E
:10345000E828A881B9810D931D932D933D938FEF9B
:103460000E9438280E943A280E943928AC81BD81E8
:103470008C938FEF0E9438280E943A280E943928A6
:10348000AA81BB818C93AA81BB810C911127222731
:10349000332740E051E060E070E00E94A527AE8154
:1034A000BF810D931D932D933D93AE81BF810D91EF
:1034B0001D912D913C91AC81BD814C915527662782
:1034C00077270E94E828AE81BF810D931D932D932D
:1034D0003D93AE81BF810D911D912D913C9140E0B6
:1034E00050E061E070E00E94A527AE81BF810D939E
:1034F0001D932D933D93AE81BF810D911D912D9113
:103500003C91A881B9814D915D916D917C910E9412
:10351000E828AE81BF810D931D932D933D9386E0E6
:10352000481A8827580A2696089584E00E9454284D
:1035300084E00E945428AC81BD810D911D912D9194
:103540003C9142E050E060E070E00E94ED28A881EC
:10355000B9810D931D932D933D93AEE6B0E00C9190
:10356000112722273327A881B9814D915D916D9153
:103570007C910E94A527AA81BB810D931D932D9359
:103580003D93AA81BB810D911D912D913C91A5E7A1
:10359000B0E04D915D916D917C910E94E828AA81E7
:1035A000BB810D931D932D933D9300917D000B30B6
:1035B00011F40C94ED1AAA81BB810D911D912D91EE
:1035C0003C9140E250E060E070E00E94E828AA816F
:1035D000BB810D931D932D933D93AA81BB810D91CA
:1035E0001D912D913C91AE81BF810D931D932D9323
:1035F0003C9388E0481A8827580A2496089584E066
:103600000E94542882E00E94542800917D000B30D3
:1036100011F00C94431BAC81BD810D911D912D9136
:103620003C9140E850E060E070E00E94AA27A3EDE2
:10363000B0E04D935D936D937D93AC81BD810D9111
:103640001C9140E850E00E944527A881B9810D9364
:103650001C93A881B9810D911C9144E050E00E9417
:103660005F27A881B9810D931C93A881B9810D9121
:103670001C9144E050E0040F151FA881B9810D93FF
:103680001C930C94791BAC81BD810D911D912D91E2
:103690003C9140E051E060E070E00E94AA27A3ED79
:1036A000B0E04D935D936D937D93AC81BD810D91A1
:1036B0001C9140E051E00E944527A881B9810D93FB
:1036C0001C93A881B9810D911C9142E050E00E94A9
:1036D0005F27A881B9810D931C93A881B9810D91B1
:1036E0001C9142E050E0040F151FA881B9810D9391
:1036F0001C93A3EDB0E00D911D912D913C91A9E794
:10370000B0E04D915D916D917C910E94E828A3ED10
:10371000B0E00D931D932D933D93A3EDB0E00D917B
:103720001D912D913C91ACE6B0E04D915C916627E6
:1037300077270E94E828A3EDB0E00D931D932D9309
:103740003D930E94B81FA881B981AD90BC90A7EFAE
:10375000B0E0AA0DBB1D8C91AA81BB818D938827F7
:103760008D938D938C93A881B9810E940D27AA8196
:10377000BB810D911D912D913C9140E051E060E0A5
:1037800070E00E94A527AA81BB810D931D932D9304
:103790003D93AA81BB810D911D912D913C91A881F2
:1037A000B981AD90BC90A7EFB0E0AA0DBB1D4C91C4
:1037B0005527662777270E94E828AA81BB810D93A9
:1037C0001D932D933D9300917D000B3011F00C94CF
:1037D000491CA881B9810E940D27AA81BB810D9146
:1037E0001D912D913C9140E051E060E070E00E941D
:1037F000A527AA81BB810D931D932D933D93AA818B
:10380000BB810D911D912D913C91A881B981AD9005
:10381000BC90A7EFB0E0AA0DBB1D4C9155276627C1
:1038200077270E94E828AA81BB810D931D932D93D1
:103830003D93A881B9810E940D27AA81BB810D917A
:103840001D912D913C9140E051E060E070E00E94BC
:10385000A527AA81BB810D931D932D933D93AA812A
:10386000BB810D911D912D913C91A881B981AD90A5
:10387000BC90A7EFB0E0AA0DBB1D4C915527662761
:1038800077270E94E828AA81BB810D931D932D9371
:103890003D93AA81BB810D911D912D913C91AE81EB
:1038A000BF810D931D932D933C9386E0481A882782
:1038B000580A2496089581E00E94542881E00E94CD
:1038C00054288FEFAA81BB818C9380E0A881B981B5
:1038D0008C93A881B9810C91073018F011F00C94E9
:1038E0007E1C91E0AA81BB810E942728A881B98112
:1038F0008C918F5F8C9311F00C94691C82E0481AB4
:103900008827580A2496089581E00E94542881E06F
:103910000E94542881E00E94542882E00E9454288A
:1039200082E00E9454288FEFAA85BB858C9381E0AA
:10393000A885B9858C93A885B9850C91003418F0B9
:1039400011F00C94AD1C0E945B1CA885B9858C916C
:103950008F5F8C9311F00C949B1CC49881E0A88518
:10396000B9858C93A885B9850C91003418F011F0B5
:103970000C94C41C0E945B1CA885B9858C918F5F38
:103980008C9311F00C94B21C8AE090E00E944528C0
:10399000A895EE81FF81FA93EA935A924A9280E4C5
:1039A000A42DB52D8C9381E00E94F4265A924A9260
:1039B00000E010E020E030E0A42DB52D0D931D9324
:1039C0002D933C9384E00E94F4260E949522269633
:1039D00085E00E94F026AE81BF810C91013011F488
:1039E0000C94FB1CC49AE6EFF4E50E948C270E941D
:1039F00098270C94B21F81E0AA85BB858C93A8956B
:103A000080E090E0A881B9818D939C93EE81FF8145
:103A1000FA93EA935A924A9281E4A42DB52D8C939D
:103A200081E00E94F4265A924A9200E010E020E0E1
:103A300030E0A42DB52D0D931D932D933C9384E080
:103A40000E94F4260E949522269685E00E94F02688
:103A5000A881B9810E940727AE81BF810C910030F7
:103A600081E009F080E08F93A881B9810D911C91CC
:103A7000003050E0150781E009F080E09F91892B2C
:103A8000882311F40C94061DC49AA881B9810D9164
:103A90001C91003050E0150711F00C94571DEEEF0B
:103AA000F4E50E948C270E9498270C94B21FA895D9
:103AB00084E690E00E944528A895C49881E090E0B3
:103AC0000E944528EE81FF81FA93EA935A924A9226
:103AD00080E5A42DB52D8C9381E00E94F4265A92A6
:103AE0004A9201E010E020E030E0A42DB52D0D93C6
:103AF0001D932D933C9384E00E94F4260E9495220E
:103B0000269685E00E94F02685E090E00E944528F8
:103B1000C49A8AE090E00E944528A89500E010E051
:103B200020E030E0A9E7B0E00D931D932D933C9386
:103B300000E010E020E030E0A3EDB0E00D931D9335
:103B40002D933C930E94B81F00E010E020E030E08D
:103B5000A3EDB0E00D931D932D933C930027AEECA5
:103B6000B0E08C9187FB0EF401E041E0041711F006
:103B70000C94BC1D0C94B21FA89500910401023056
:103B800011F40C94501E8091BA0280937D00A1EC38
:103B9000B2E00D91112740E051E00E945F27AA8119
:103BA000BB810D931C93AA81BB810D911C91A0EC4C
:103BB000B2E04D915527040F151FAA81BB810D93CB
:103BC0001C93AA81BB810D911C912227332740E0D1
:103BD00050E061E070E00E94A527A9E7B0E00D93F6
:103BE0001D932D933D93AFEBB2E00D91112740E073
:103BF00051E00E945F27AA81BB810D931C93AA818B
:103C0000BB810D911C91AEEBB2E04D915527040F95
:103C1000151FAA81BB810D931C93A9E7B0E00D91FC
:103C20001D912D913C91AA81BB814D915C9166279C
:103C300077270E94E828A9E7B0E00D931D932D9304
:103C40003D9300917D000C3011F00C942A1E8BE006
:103C500080937D0000917D000E3011F00C94331E96
:103C60008BE080937D0000917D000F3011F00C946B
:103C70003C1E8BE080937D00A9E7B0E00D911D9183
:103C80002D913C91A3EDB0E00D931D932D933C93AA
:103C90000E94B81FA3EDB0E00E9413270C94A41E4D
:103CA00000912E01063411F00C947A1E84E080936A
:103CB0007D0087E3A885B9858C93A885B9850C918B
:103CC0000C3318F011F00C94781EA885B985AD90CE
:103CD000BB24A7EFB0E0AA0DBB1D8C910E949B27CF
:103CE000A885B9858C918F5F8C9311F00C945D1E23
:103CF0000E94982700914A01063411F00C94A41EEA
:103D00008BE080937D0083E5A885B9858C93A88599
:103D1000B9850C91073518F011F00C94A21EA885F6
:103D2000B985AD90BB24A7EFB0E0AA0DBB1D8C9167
:103D30000E949B27A885B9858C918F5F8C9311F089
:103D40000C94871E0E949827E8E0F5E50E948C27D6
:103D5000A8E6B7E0EDE7F0E00E9414290E9484276E
:103D60000E949827EAE1F5E50E948C27A8E6B7E0D3
:103D7000E9E7F0E00E9408290E9484270E94982722
:103D800084E0A885B9858C93A885B9850C910B3002
:103D900018F011F00C94DF1EA885B985AD90BB24F6
:103DA000A7EFB0E0AA0DBB1D8C910E949B27A885B0
:103DB000B9858C918F5F8C9311F00C94C41E0E9476
:103DC00098278091050180936E00ECE2F5E50E9452
:103DD0008C27A8E6B7E0EEE6F0E00E9414290E94E6
:103DE00084270E94982700916E00003011F00C94F7
:103DF000FB1E0C94B21F00916E00003418F011F0FD
:103E00000C94041F0C94061F0C94B21F80910601A1
:103E1000AE81BF818C9380910701AC81BD818C9371
:103E2000AC81BD819C91AE81BF818C91ACE6B0E04C
:103E30008D939C9380910E01AE81BF818C93809174
:103E40000F01AC81BD818C93AC81BD819C91AE8111
:103E5000BF818C91AFE6B0E08D939C93AFE6B0E06C
:103E60000D911C91003050E0150711F00C944E1F7D
:103E700080911C01AE81BF818C9380911D01AC812A
:103E8000BD818C93AC81BD819C91AE81BF818C91B1
:103E9000AFE6B0E08D939C930C944E1FAFE6B0E07C
:103EA0000D911C91003050E0150711F00C945A1F31
:103EB0000C94B21F02E010E020E030E0AFE6B0E08A
:103EC0004D915C91662777270E94A527A1E7B0E076
:103ED0000D931D932D933D93A1E7B0E00D911D919E
:103EE0002D913C91ACE6B0E04D915C91662777272F
:103EF0000E94E828A1E7B0E00D931D932D933D9318
:103F0000A1E7B0E00D911D912D913C91A3EDB0E0A2
:103F10004D915D916D917C910E94E828A1E7B0E000
:103F20000D931D932D933D93ECE3F5E50E948C27B3
:103F3000A8E6B7E0E1E7F0E00E9408290E948427A4
:103F40000E949827A1E7B0E00D911D912D913C9121
:103F5000A3EDB0E00D931D932D933C9380E0AA85D3
:103F6000BB858C9387E0481A8827580A2A960895BB
:103F700081E00E94542881E00E94542882E00E943F
:103F8000542882E00E9454288FEFAE81BF818C9329
:103F900091E0AE81BF810E94272891E0AE81BF8170
:103FA0000E94272891E0AE81BF810E94272891E0DE
:103FB000AE81BF810E94272891E0AE81BF810E941F
:103FC000272891E0AE81BF810E94272891E0AE8131
:103FD000BF810E94272891E0AE81BF810E942728DF
:103FE00091E0AE81BF810E94272891E0AE81BF8120
:103FF0000E94272891E0AE81BF810E94272891E08E
:10400000AE81BF810E94272891E0AE81BF810E94CE
:10401000272891E0AE81BF810E94272891E0AE81E0
:10402000BF810E94272891E0AE81BF810E9427288E
:10403000C49880E090E0A881B9818D939C938FEF24
:104040000E9438280E943A280E943928AE81BF81F8
:104050008C93A881B9810E940727AE81BF810C9102
:10406000003081E009F480E08F93A881B9810D913F
:104070001C91003050E0150781E009F080E09F912D
:10408000892B882311F40C941F20A881B9810D91EC
:104090001C91003050E0150711F00C945C20E4E412
:1040A000F5E50E948C270E9498277091CE007068D9
:1040B0007093CE000C94A921EE81FF81FA93EA93CC
:1040C0005A924A9281E5A42DB52D8C9381E00E94ED
:1040D000F4265A924A92A3EDB0E00D911D912D91D4
:1040E0003C91A42DB52D0D931D932D933C9384E00D
:1040F0000E94F4260E949522269685E00E94F026D2
:104100000027AEECB0E08C9187FB0EF401E041E0BB
:10411000041711F00C949C20E2E5F5E50E948C2731
:10412000A8E6B7E0E3EDF0E00E9408290E948427AA
:104130000E9498270C94A921A895AE81BF810C916B
:10414000003011F00C94E72080E090E0A881B98164
:104150008D939C938FEF0E9438280E943A280E94EA
:104160003928AE81BF818C93A881B9810E9407272D
:10417000AE81BF810C91003081E009F480E08F9323
:10418000A881B9810D911C91003050E0150781E0A4
:1041900009F080E09F91892B882311F40C94AA20C8
:1041A000A881B9810D911C91003050E0150711F0E4
:1041B0000C94E720ECE6F5E50E948C270E949827F6
:1041C0007091CE0070687093CE000C94A921AE81DE
:1041D000BF810C910F3F11F00C94312180E090E0F1
:1041E000A881B9818D939C938FEF0E9438280E94FB
:1041F0003A280E943928AE81BF818C93A881B98169
:104200000E940727AE81BF810C910F3F81E009F426
:1042100080E08F93A881B9810D911C91003050E00E
:10422000150781E009F080E09F91892B882311F424
:104230000C94F420A881B9810D911C91003050E0BC
:10424000150711F00C943121EAE7F5E50E948C275F
:104250000E9498277091CE0070687093CE000C94E5
:10426000A921AE81BF810C910E3F11F40C944E2117
:10427000E8E8F5E50E948C27A8E6B7E0EE81FF812B
:104280000E9414290E9484270E949827C49A709142
:10429000CE0070687093CE000C94A92180E090E06D
:1042A000AA81BB818D939C9380E0AE81BF818C936A
:1042B000AE81BF810C910F3F18F011F00C9490214A
:1042C000AA81BB810E9407278FEF0E9438280E9495
:1042D0003A280E943928AA81BB81AD90BC90A7EFF3
:1042E000B0E0AA0DBB1D8C93AA81BB810E94072759
:1042F0008FEF0E9438280E943A280E943928AA810C
:10430000BB81AD90BC90A7EFB0E0AA0DBB1D8C9314
:10431000AE81BF818C918F5F8C9311F00C945821EA
:104320008FEF0E9438280E943A280E943928AE81D7
:10433000BF818C938FEF0E9438280E943A280E94F8
:104340003928AE81BF818C93C49AA3EDB0E00E945E
:10435000F82686E0481A8827580A2896089582E0A9
:104360000E94542881E00E94542880E0AE81BF81E1
:104370008C930E945B1CC49880E090E0AA81BB8172
:104380008D939C938FEF0E9438280E943A280E94B8
:104390003928A881B9818C93AA81BB810E94072703
:1043A000A881B9810C91003081E009F480E08F93FD
:1043B000AA81BB810D911C91003050E0150781E06E
:1043C00009F080E09F91892B882311F40C94C2217D
:1043D000AA81BB810D911C91003050E0150711F0AE
:1043E0000C94FF21E4E4F5E50E948C270E949827B5
:1043F0007091CE0070687093CE000C948F22E8818B
:10440000F981FA93EA935A924A9281E5A42DB52D47
:104410008C9381E00E94F4265A924A92AA85BB8529
:104420000D911D912D913C91A42DB52D0D931D93B2
:104430002D933C9384E00E94F4260E9495222696B8
:1044400085E00E94F026A881B9810C91003011F01E
:104450000C94562280E090E0AA81BB818D939C93BE
:104460008FEF0E9438280E943A280E943928A8819C
:10447000B9818C93AA81BB810E940727A881B98149
:104480000C91003081E009F480E08F93AA81BB8118
:104490000D911C91003050E0150781E009F080E09B
:1044A0009F91892B882311F40C943022A881B98123
:1044B0000C910F3F11F00C94892280E090E0AA81CA
:1044C000BB818D939C938FEF0E9438280E943A28DD
:1044D0000E943928A881B9818C93AA81BB810E944E
:1044E0000727A881B9810C910F3F81E009F480E092
:1044F0008F93AA81BB810D911C91003050E015076C
:1045000081E009F080E09F91892B882311F40C94BD
:104510006322A881B9818C91AE81BF818C9383E0A5
:10452000481A8827580A2496089584E00E9454283F
:1045300081E00E94542882E00E9454288FEFAA81D3
:10454000BB818C9391E0AA81BB810E94272891E0D6
:10455000A885B9850E942728AE81BF810D911D9144
:104560002D913C9140E052E060E070E00E94A52770
:10457000AC81BD810D931D932D933D93AC81BD8185
:104580008F9314968E910E941B238E910E941B2361
:104590008E910E941B238E910E941B2385E90E940D
:1045A0001B238F9180E090E0A881B9818D939C932B
:1045B0008FEF0E9438280E943A280E943928AA8149
:1045C000BB818C93A881B9810E940727AA81BB81F6
:1045D0000C910F3F81E009F480E08F93A881B981AD
:1045E0000D911C91003050E0150781E009F080E04A
:1045F0009F91892B882311F40C94D822A881B9812A
:104600000D911C91003050E0150711F00C9413230C
:10461000E6E9F5E50E948C270E9498277091CE006C
:1046200070687093CE00AA81BB818C91AA85BB85EE
:104630008C930C9420238FB9779BFECF8FB1089574
:1046400087E0481A8827580A269608955A924A926F
:1046500084E298E0A42DB52D8D939C9382E00E9476
:10466000F4265A924A9280E0A42DB52D8C9381E0D5
:104670000E94F4260E949F25249683E00E94F02643
:10468000EF93FF93ECE8F1E00E941928FF91EF917E
:10469000BB27A0E38C9182FBDEF789E190E00E94CA
:1046A00045285A924A9280E298E0A42DB52D8D9328
:1046B0009C9382E00E94F4265A924A9280E0A42DB4
:1046C000B52D8C9381E00E94F4260E949F252496AC
:1046D00083E00E94F02689E190E00E9445280E9434
:1046E0002724089582E00E94542800E011E0AA8166
:1046F000BB814D9155270E945F27A881B9810D93F9
:104700001C93A881B9810D911C91AA81BB814D9107
:104710005527040F151FA881B9810D931C935A9238
:104720004A92AA81BB818D919C91A42DB52D8D9328
:104730009C9382E00E94F4265A924A928BE0A42D28
:10474000B52D8C9381E00E94F4260E949F2524962B
:1047500083E00E94F0265A924A9280E298E0A42DCB
:10476000B52D8D939C9382E00E94F4265A924A9232
:1047700080E0A42DB52D8C9381E00E94F4260E9448
:104780009F25249683E00E94F02682E0481A88271D
:10479000580A2296089582E00E94542800E110E011
:1047A000AC81BD814D9155270E945F27A881B981B9
:1047B0000D931C93A881B9810D911C91AA81BB8195
:1047C0004D915527040F151FA881B9810D931C9396
:1047D0005A924A92AA81BB818D919C91A42DB52DAC
:1047E0008D939C9382E00E94F4265A924A9282E032
:1047F000A42DB52D8C9381E00E94F4260E949F2564
:10480000249683E00E94F02682E0481A8827580AFE
:10481000229608955A924A92AA81BB818D919C91C9
:10482000A42DB52D8D939C9382E00E94F4265A927C
:104830004A9283E0A42DB52D8C9381E00E94F4264A
:104840000E949F25249683E00E94F026089581E02F
:104850000E94542881E00E945428C49AD898C29893
:1048600080E0A881B9818C9380E0AA81BB818C9380
:10487000AA81BB810C910F3118F011F00C945C24CB
:1048800091E0A881B9810E94272891E0A881B9818F
:104890000E94272891E0A881B9810E94272891E0F1
:1048A000A881B9810E942728AA81BB818C918F5F42
:1048B0008C9311F00C943824C29AD89A82E0481A4A
:1048C0008827580A2496089581E00E9454285A9215
:1048D0004A9280E298E0A42DB52D8D939C9382E0BE
:1048E0000E94F4265A924A9280E0A42DB52D8C9312
:1048F00081E00E94F4260E949F25249683E00E9476
:10490000F026AA81BB810C91003011F00C94972401
:104910005A924A9280E0A42DB52D8C9381E00E949A
:10492000F4260E941125229681E00E94F026AA8199
:10493000BB810C91013011F00C94AD245A924A9233
:1049400085E6A42DB52D8C9381E00E94F4260E946B
:104950001125229681E00E94F026AA81BB810C914C
:10496000023011F00C94DA245A924A9283E6A42D74
:10497000B52D8C9381E00E94F4260E941125229689
:1049800081E00E94F02688EC90E00E9445285A922F
:104990004A9280E0A42DB52D8C9381E00E94F426EC
:1049A0000E941125229681E00E94F02682E390E089
:1049B0000E944528AA81BB810C91033011F00C9410
:1049C00003255A924A9282E6A42DB52D8C9381E05C
:1049D0000E94F4260E941125229681E00E94F02672
:1049E00080E991E00E9445285A924A9280E0A42DE5
:1049F000B52D8C9381E00E94F4260E941125229609
:104A000081E00E94F0268AE090E00E9445288AE03A
:104A100090E00E94452881E0481A8827580A22968B
:104A2000089581E00E945428C49AD898C298AA8117
:104A3000BB810C91003018F011F00C9421250C94DE
:104A40005B2583E5A881B9818C9391E0A881B98128
:104A50000E9427288FEEA881B9818C9391E0A881CC
:104A6000B9810E9427288EE6A881B9818C9391E0B4
:104A7000A881B9810E94272891E0AA81BB810E9468
:104A8000272880E0A881B9818C9391E0A881B98121
:104A90000E94272891E0A881B9810E94272891E0EF
:104AA000A881B9810E94272891E0A881B9810E943C
:104AB00027280C94972585E4A881B9818C9391E0EF
:104AC000A881B9810E94272888E7A881B9818C93A1
:104AD00091E0A881B9810E94272889E6A881B9813F
:104AE0008C9391E0A881B9810E94272884E7A8814E
:104AF000B9818C9391E0A881B9810E94272880E038
:104B0000A881B9818C9391E0A881B9810E9427285E
:104B100091E0A881B9810E94272891E0A881B981FC
:104B20000E94272891E0A881B9810E942728C29A73
:104B3000D89A81E0481A8827580A2296089581E079
:104B40000E945428C29AD8985A924A9282E0A42D80
:104B5000B52D8C9381E00E94F4260E945426229663
:104B600081E00E94F0265A924A92AC81BD818C91DC
:104B7000A42DB52D8C9381E00E94F4260E9454262A
:104B8000229681E00E94F026AC81BD8111968C9125
:104B9000A881B9818C935A924A92AA81BB818C9147
:104BA000A42DB52D8C9381E00E94F4260E945426FA
:104BB000229681E00E94F026AC81BD818C91A88173
:104BC000B9818C935A924A92AA81BB818C91A42D6F
:104BD000B52D8C9381E00E94F4260E9454262296E3
:104BE00081E00E94F026D89A81E0481A8827580A66
:104BF0002296089581E00E94542881E00E94542862
:104C000082E00E945428C29AD8985A924A9283E02D
:104C1000A42DB52D8C9381E00E94F4260E94542689
:104C2000229681E00E94F0265A924A92A885B98580
:104C30008C91A42DB52D8C9381E00E94F4260E94C6
:104C40005426229681E00E94F026EC81FD81FA93A1
:104C5000EA930E945A262296EA81FB81FA93EA930C
:104C60000E945A262296D89AAC81BD810D911127B7
:104C700040E051E00E945F27A881B9810D931C9309
:104C8000A881B9810D911C91AA81BB814D915527B5
:104C9000040F151FA885B9850D931C9384E0481A4D
:104CA0008827580A2696089591E0A881B9810E9424
:104CB0002728089581E00E94542891E0A881B981B5
:104CC0000E941C28A881B9818C91AA81BB818C93F8
:104CD00081E0481A8827580A2296089582E00E94A7
:104CE000542881E00E945428C49ABB27A0E38C91E9
:104CF00082FBDEF7C298AC81BD810D911C91003022
:104D000052E0150711F00C94BD2681E090E0AA81D5
:104D1000BB818D939C9380E0A881B9818C93A881FD
:104D2000B9810C910F3018F011F00C94BB26BB2701
:104D3000A0E38C9182FBDEF790E2AA81BB81AD906B
:104D4000BC90A7EFB0E0AA0DBB1D0E942728AA8146
:104D5000BB810D911C9140E250E0040F151FAA8108
:104D6000BB810D931C93A881B9818C918F5F8C932B
:104D700011F00C948F260C94E92681E090E0AA8132
:104D8000BB818D939C93AC81BD814D915C91AA8137
:104D9000BB810D911C910417150718F011F00C94AC
:104DA000E926BB27A0E38C9182FBDEF7C29A91E053
:104DB000AA81BB81AD90BC90A7EFB0E0AA0DBB1D4E
:104DC0000E942728AA81BB810E94072711F00C941A
:104DD000C326C29A83E0481A8827580A2496089561
:104DE000481A8827580A0895480E8827581E08959B
:104DF0000D911D912D913C9181E0080F8827181F7E
:104E0000281F381F3C932E931E930E930895ED9107
:104E1000FC913196FC93EE930895ED91FC913197BE
:104E2000FC93EE9308950D911D912D913C910150AD
:104E30001040204030403C932E931E930E930895D3
:104E400008D03DD000FC10D0089503D01ED001F84A
:104E5000F9CF0024E89457FF02C009D0689400F805
:104E60000BD010F80124089502D009D00895509570
:104E700040954F5F5F4F0895E89417FF08950095A0
:104E800010950F5F1F4F68940895352F242FE894D5
:104E9000452B11F468940895512F402F00271127B6
:104EA00080E1440F551F001F111F021B130B4160AF
:104EB00018F4020F131F4E7F8A9599F708950F92E9
:104EC000049F202C312C419F300C509F030C022D4D
:104ED000102D0F900895C8950D9231960020D9F7A6
:104EE00008958F938D918823E9F711978F910895F5
:104EF00081E05F9B8827089588275F9B089500C005
:104F00005F9BFECF8CB10895A8E6B7E08D91882312
:104F100011F011D0FBCF08950E948A28802D11F046
:104F20000AD0FACF08958D9106D03A95E1F7089509
:104F30008DE001D08AE05D9BFECF8CB9089588EEAC
:104F400093E0A3D03197D9F7089550D00AD000FC50
:104F500005D008954BD020D001F8F9CF52D05AD0C7
:104F60000895842F952FA62FB72F442755276627FE
:104F70007727F1E2889409C020F4480F591F6A1F6F
:104F80007B1F769567955795479537952795179584
:104F90000795FA9589F70895842F952FA62FB72F97
:104FA000E894452B462B472B11F468940895402F25
:104FB000512F622F732F0027112722273327F0E26A
:104FC000440F551F661F771F001F111F221F331F1D
:104FD000081B190B2A0B3B0B416028F4080F191F03
:104FE0002A1F3B1F4E7FFA9559F708950024E89435
:104FF00077FF02C006D0689400F809D010F80124A9
:10500000089512D04F5F5F4F6F4F7F4F0895E89420
:1050100037FF089500951095209530950F5F1F4F2D
:105020002F4F3F4F68940895409550956095709527
:1050300008953197F1F708950E9438288C910E94C5
:105040003A288D939A95D1F70E94392808950E94A5
:1050500038288D910E943A289A95D9F70E943928CC
:105060000895BF9ABE98C69ABD9A80E58DB90895F5
:10507000089508958FB9779BFECF8FB108956894F6
:1050800062F80895E89462F80895EF93FF93EE278D
:10509000E82BE92B31F0E0EDF7E03197F1F70197DC
:1050A000D1F7FF91EF9108955A924A92480E8827BE
:1050B000581E089599910027A90FB01F1197492FE5
:1050C0004A955E2F6F2FE89411274395203019F0F1
:1050D000C895802D01C080818823B9F07C91772309
:1050E000A1F0781739F40EF0042F139568941196F7
:1050F0003196EBCF112321F0411BA11B1127B10BDE
:10510000E894E52FF62F1196E0CF882311F00027C1
:1051100008950895C895319600200895819104D08E
:105120008D938823D9F70895813418F0823608F4D6
:1051300080620895819104D08D938823D9F70895D2
:10514000813618F08B3708F48F7D089580E30EF4D4
:10515000839508952E2E3F2E992781918D3209F047
:1051600093958823D1F79A95E22DF32D112361F0C1
:10517000091718F011F0101B01C0191B28F021F0BD
:1051800080E28D931A95E9F780818D3219F48D9321
:10519000319604C0222311F08BE28D93091738F069
:1051A00031F0091B21F080E38D930A95E9F7819195
:1051B0008D938823E1F7332351F0EA2FFB2F3196AB
:1051C00033958E9182933A95E1F78EE28C93089510
:1051D000040F151F261F371F0895041B150B260BE0
:1051E000370B089504171507260737070895000F92
:1051F000111F221F331F089500951095209530959B
:105200000F5F1F4F2F4F3F4F0895019110810EC028
:1052100001911191219130810BC00191108117FFF3
:1052200005C03FEF2FEF04C000811127222733274D
:1052300037FF03C0E1DF8DE28D93CF93DF93CF92F1
:10524000DF92EF92AA24BB24CC24DD24EE2440E29A
:10525000CAE0DD2755E093E38881890F87FD9F70C1
:1052600083FD907F891B89935A95A9F7C0DFAA1CFB
:10527000BB1CCC1CDD1CEE1C4A9551F7E894EFE0FA
:10528000FF2782910ED0EB30E0F71EF068948A2D54
:105290000CD088278D93EF90DF90CF90DF91CF9146
:1052A0000895982F829501D0892F8F70805D26F008
:1052B000803309F4089568948D9308950027112789
:1052C000222733271DD08A3328F4803318F005D0E5
:1052D00015D0F9CF0EF490CF089580538F93402FBF
:1052E000512F622F732F83DF82DF72DF80DF8F9178
:1052F0009927080F191F291F391F08958D910895A7
:10530000E894FCDF8032E9F38B32D9F38930C9F3BA
:105310008D3211F46894F2CF089588278D93089503
:1053200081918D938823E1F7089581918032E9F38B
:10533000F8CFF6DF11978E918032E9F31196EDCF19
:10534000F4DFF8CF09919191992351F08A95D9F71B
:10535000319781918D930A9519F08823D1F708959B
:10536000DCCFE199FECFEEBBFFBB3196089591E013
:1053700001C092E07B3751F47FB7F894F2DF8D9152
:105380008DBBE29AE19A9A95C9F77FBF7727089576
:1053900091E001C092E0E5DFE09A8DB38D939A959C
:1053A000D1F70895FF93881BF9E0001FFA9511F4D7
:1053B000FF910895881F841B18F4840F8894F5CFFB
:1053C0000894F3CF689401C0E894AF93BF938D9194
:1053D00016F0919103C00E948A28902D891718F029
:1053E00011F48823A1F7BF91AF9108954D50335325
:1053F00054414D50205265616C6974792D53797315
:1054000020342E35490053005000454570726F6DB1
:1054100020002C004D4D4320696E69742000726598
:10542000747279202E2E2E0044535020696E6974B8
:1054300020004F005A004800210059004E00420051
:1054400058004400450056004D00540049004C00EF
:10545000636F6E6669672073656172636800434FAE
:105460004E4649470000636F6E66696720666F7538
:105470006E6400006E6F7420666F756E64003B0092
:105480005B005D3D0000766F6C00766F6C756D653E
:105490003A00696E7000696E707574733A006C63DF
:1054A0006B006C6F636B65643A006E756D006E75B2
:1054B0006D66696C653A0000696E7400696E7465AA
:1054C00072727570743A00006C6F70006C6F6F7060
:1054D0003A00616C6C00616C6C3A0000636E7400A1
:1054E000636E743A00004D5033006F6B0000200073
:1054F000442000002E004E6F206361726400426100
:105500006420636172640000506172746974696F31
:105510006E2074797065203A00005061727469746D
:10552000696F6E2073746172743A0000536563741E
:105530002F636C757374657220203A00526F6F741C
:10554000203A000052656164206572726F722031EA
:10555000000052656164206572726F722032206FA4
:105560006E20736563746F723A2000005265616447
:10557000206572726F72203300005265616420658D
:1055800072726F722034000052656164206572721D
:105590006F7220352000526561642074696D656FFB
:0455A000757400001E
:00000001FF
